:020000020000FC
:080000000C94CE010C94CC001D
:040014000C944B01FC
:040034000C948A019D
:040040000C94F80024
:040048000C94770C91
:100050000C94460CBF93AF93A8E8B1E016E02D9145
:100060003D91232B31F016961A95C9F7EF91FF9128
:1000700016C0ED93FD93ED920D93EF91FF910191D9
:100080000D9301910D9318973297ED93FC93E831FE
:1000900029F4F13019F40BA100640BA31197089512
:1000A0000A2F0B2B89F0ED91FD9114960D911D9166
:1000B00001931193EA3131F4F13021F40BA10F7B5C
:1000C0000BA3C8D7189701D00895FD92FD92FD9219
:1000D000FD92FD92FD92FD92FD92089507E0A8E841
:1000E000B1E0F3DF0A95E9F70895A8E8B1E026E06A
:1000F000BF93AF930D911D91012B21F012972F9378
:1001000009952F91AF91BF9118962A9589F7089577
:100110000D911D9112962D913C913F3F19F03A950A
:100120003C9389F0322F319533953E93222321F071
:10013000D801FD92FD920DC012972D913D91D801ED
:100140002D933D9306C01597FF93EF93A9DFEF9191
:10015000FF9108954A2F4B2B59F04D914E1741F4C2
:100160004D914F1729F40D931D9312960D931D93E6
:100170000895E8E8F0E0B9DF08955A9A0E94ED0C7E
:1001800002E01E8510FD03E00093690001D0089590
:10019000E89A0895E89808950F930FB70F93946025
:1001A0000F910FBF0F9118950F93F4BC05E005BD9B
:1001B0000F910895BF93AF93ADE7B0E0AF8FB8A3B1
:1001C000AF91BF910895FF8EF8A208950F93FF8E0F
:1001D000F8A201E005BB01E806BD01E000936E0056
:1001E0000F9108950F9300E000936E000F91089512
:1001F0000F9301E806BD78940FB70F931F93BF9339
:10020000AF93AF8DB8A10A2F0B2B51F01197AF8F81
:10021000B8A331F400910502002311F49860FCA208
:100220000DA1000F1E2D4F9B1127012B0DA3003890
:1002300049F40CA10E15A1F00BA108600BA3ECA2D0
:10024000B9DF0EC00F3721F00F3F51F413D008C0B3
:100250000CA1002329F09062FCA20BA1077F0BA345
:10026000AF91BF911F910F910FBF0F9118950CD0B7
:10027000ADDF0895B7DF01D0089510E810936D0049
:1002800014E010936800089510E010936D0010E0E2
:100290001093680008950F930FB71F930F93E7DF34
:1002A0000F911F910FBF0F91189504E000938100EB
:1002B0000AEF009385000AEE0093840022D008958F
:1002C000BF93AF93A8E0B7E0F894A9A3BAA378943A
:1002D000AF91BF910895BF93AF93A8E7B0E0F894B2
:1002E000A9A3BAA37894AF91BF910895F9A2FAA2F5
:1002F00008951F9309A11AA1012B09F00E2D1F913A
:10030000089501E000936F00F1DF089500E000938D
:100310006F0008950F930AEE009384000AEF009394
:10032000850078940FB71F930F93BF93AF93A9A144
:10033000BAA10A2F0B2B21F01197A9A3BAA301F49C
:100340000F81002329F00A9511F4906808850F8326
:1003500008890A9511F490640FE0088BAF91BF9162
:100360000F911F910FBF0F911895A89504B7077FA4
:1003700004BF0091600008610093600000270093B3
:1003800060000895F894A8950091600008610093BA
:1003900060000AE00093600078940895F894E5DF27
:1003A0002227E0E0F1E014E0002721930A95E9F725
:1003B0001A95D1F7C0ECD1E0FF24EE24E3949927FD
:1003C000882499240FEF0DA308AB02E30EA30FE4DA
:1003D0000FA3E8E4FBE1E0930001F0930101E8EDF5
:1003E000FCE1E0930102F0930202E0930401F09338
:1003F0000501EEEBFAE2E0933401F09335010AE4F3
:100400000093360106E019E4EFE1F1E01083349641
:100410000A95E1F7ECEBFEE1E0933C01F0933D013E
:10042000E8E8FFE1E0934001F0934101E2EDFFE1F4
:10043000E0934401F0934501EEE0F0E2E0934801DF
:10044000F0934901EAE7F0E2E0935001F0935101A3
:10045000E6E8F1E2E0935801F0935901E0E4F2E2BA
:10046000E0936001F0936101ECEAF2E2E09368014D
:10047000F0936901E4E5F3E2E0937001F093710118
:10048000E4EDF3E2E0937801F0937901E2EAF4E23B
:10049000E0938001F09381010CE308830EE30F8366
:1004A00008870FE0088BE6EFF2E0EEAFFFAF01EC5C
:1004B0000093640079DEF9DE31D10E94250D0E949F
:1004C0002B0C60D568D5D9DE09DE06D60E87C2D5DD
:1004D000F7D50D8705E00A8BF98AF5D50B8F002338
:1004E00011F00FEF098BF5D50F87F9D5098F0E9411
:1004F000180D00910302002331F40E94E00B0F3F1E
:1005000011F40E94C80AD9D50E8F002321F0F09271
:100510000401F0920501DAD50C87002311F40FE0F5
:1005200001C007E00A870987ABD742D279807ED025
:10053000C3D709810715D9F30A950983C4D11DDEF4
:10054000789422D60E94D60A1FD60E94400C6ED004
:1005500095FF19C09F7DECE1F3E0EEAFFFAFEED465
:1005600000E5E9D3A0E4B1E0DCD363D063D30FA10D
:100570000F3429F0BEDE0023C1F70FE4DCD3E6EF31
:10058000F2E0EEAFFFAF93FF26C00B85002319F515
:1005900001DE1DD50E94030D0C85002349F403E301
:1005A000B4D3A0E3B1E09DD3ACE2B1E09ED305C0EB
:1005B00006E3ABD3A0E1B1E094D338D0BED20EA114
:1005C000023329F096DE0023C1F799D327D30E9486
:1005D0000A0DDEDDFED490FDEFD5B9CFFF93EF938A
:1005E000EEADFFAD0995EF91FF9108950F921F9227
:1005F0000F931F932F933F934F936F938F93BF93BB
:10060000AF93FF93EF935F937F9310D07F915F91B0
:10061000EF91FF91AF91BF918F916F914F913F916A
:100620002F911F910F911F900F900895BAD024D051
:100630000895E0D021D008950F921F920F931F9339
:100640002F933F934F936F938F93BF93AF93FF93EA
:10065000EF935F937F93EDDF7F915F91EF91FF9138
:10066000AF91BF918F916F914F913F912F911F91BA
:100670000F911F900F90089592FF1EC01F81088553
:100680000F83011B19F00E3108F406C00D8D0023F5
:1006900011F419D101C059D11091050210FF05C004
:1006A00011FFABD412FDB0D406C0AEA5BFA50A2F72
:1006B0000B2B09F0A2D49B7F97FF08C08DD40D8D22
:1006C000002311F400D101C040D19F7796FF02C0F2
:1006D00050DD9F7B94FF21C00A890A9511F494D4C0
:1006E00005E00A8B098D002311F001E045D69F7EBD
:1006F0000BA101FF12C0198D0D8510230B8D102346
:1007000049F00B81043031F4A4E1B1E0E2E6FDE10F
:1007100000EFA0DC0BA10D7F0BA30895209A219A76
:10072000229A239A389A399A3A9A3B9A539A549A27
:10073000559A5D9A5C9A089538B1307F0895582F84
:10074000580D5B0D5B98052F5F70532B58B90295C0
:1007500005B9562F590D5C0D052F5F70532B02956F
:100760005C985C9A5B9A58B905B95C985C9A089554
:10077000562F580D5B0D5B98052F5F70532B58B9A2
:10078000029505B9582F590D5C0D052F5F70532B3D
:1007900002955C985C9A5B9A58B905B95C985C9A2A
:1007A00008951127A0E0B1E0A10FBF1DA10FBF1D4B
:1007B000A10FBF1DA10FBF1DED91FD91BD90CD906B
:1007C00013950985039510170CF013C00E2F0F2BEE
:1007D00049F385918823D1F3659145914423B1F381
:1007E0004F3F01F325912F934F932DD08F916F9110
:1007F000F4CF08951127ACE3B1E0A10FBF1DA10F05
:10080000BF1DA10FBF1DA10FBF1DED91FD91BD909B
:10081000CD90139514310CF014C00E2F0F2B59F3FB
:100820005D9A85918823C9F3659145914423A9F385
:100830004F3F09F325912F934F9305D08F916F91DF
:10084000F4CF5D9A089578DFDF01EFE9F3E0522FEE
:10085000561B08F45195042F081B08F40195051741
:1008600040F4E8EBF3E08627682786274227242711
:100870004227481730F484274827842762272627F1
:100880006227442E481A522E561A08F451942224F4
:1008900033246624621710F4639401C06A944817E5
:1008A00078F05D980995250C3F1C722D720D74151A
:1008B0003F041CF0660D24183F088395481790F7F5
:1008C000FD015D9A08950F921F921F930F932F932E
:1008D0003F93FF93EF9359D31981139519831C33D9
:1008E00041F00A8D002311F0FA8E25C06BD0B3D0F1
:1008F00023C090611E85112321F4E9D510D1C0D504
:100900001AC0F9821A8113951A831C337CF01BA13B
:1009100012601BA3FA821B8113951B8300D11B81DC
:10092000183124F0FB82E092040205C01C8D1123D3
:1009300011F4EAD5A5D53DD0EF91FF913F912F91CC
:100940000F911F911F900F9008951E85112339F16B
:100950001CD308850F8319811A9519831F3F41F015
:100960000A8D002311F0FA8E19C02CD074D017C054
:100970001BE3198390611A811A951A831F3F71F442
:100980001BE31A831BA112601BA31B811A951B83F7
:10099000C6D01B811F3F11F417E11B830AD00895B5
:1009A0001C8D0D8D102B19F492D503D00895089548
:1009B0008ED5B5D003D03AD098D0089503D010D0BA
:1009C0001DD00895EAE5F5E2098115E0019FE00DEB
:1009D000F11D8F01E8E0F1E0008311839BD10895C0
:1009E000E6E8F6E20A8119E0019FE00DF11D8F01B2
:1009F000ECE0F1E0008311838DD10895E2EAF8E2A2
:100A00000A811CE0F0D60F930B81EDD6022F25E072
:100A1000029F1F91100D29E0129FE00DF11D8F0123
:100A2000E0E1F1E00083118375D1089514D029D05D
:100A30003ED00895000FE00FFF1D05911491000FA7
:100A4000111F0895EEE1FBE2F5DF08950F851EE327
:100A500000FD1AE408950981E9D6F4DFE0E2F1E04F
:100A60000083118357D1F2DF185B1283022FEADF74
:100A7000ECE1F1E0008311834DD1E8DF1C5A1283D1
:100A800008950A81D3D6DEDFE8E2F1E00083118326
:100A900041D1DCDF185D1283022FD4DFE4E2F1E004
:100AA0000083118337D1D2DF1C5C128308950B8140
:100AB0000F8400FC05C0ECE0FCE2E00FFF1D049198
:100AC000B5D6C0DFE0E3F1E00083118323D1BEDFC0
:100AD000195F1283022FB6DFECE2F1E0008311838D
:100AE00019D1B4DF1C5E128308950F85002369F4C9
:100AF000EAEEFAE20B810C3014F0E2E0FBE2E09364
:100B00003801F09339010EE305C0F0923801F092FC
:100B100039010AE400933A01009336010895E8EDA3
:100B2000FCE1E0930102F09302020E8D002321F418
:100B3000E0930401F093050108950EA1033389F4B5
:100B400095FF03C09F7D92D474C093FF72C004E3ED
:100B5000DCD0D5D0A8E2B1E0C4D0A4E2B1E0C5D0E9
:100B600068C0043389F495FF03C09F7D75D461C0CC
:100B700093FF5FC005E3C9D0C2D0A0E2B1E0B1D01D
:100B8000ACE1B1E0B2D055C0053359F495FF03C0D4
:100B90009F7D58D44EC093FF4CC009E3B6D0AFD070
:100BA00029C0063369F495FF03C09F7D5FD441C01F
:100BB00093FF3FC007E3A9D0ACE0B1E092D039C0C9
:100BC000073369F495FF03C09F7D46D432C093FF7D
:100BD00030C008E39AD0A8E0B1E083D02AC008333F
:100BE00099F495FF03C09F7D2DD423C093FF21C0AE
:100BF00009E38BD0A8E0BEE1A0931401B0931501E6
:100C0000A4E1B1E06ED015C0093309F007C095FF2B
:100C100003C09F7D79D404C093FF0BC058D4C9DEB4
:100C200068D0A0E0B0E0A0931401B093150102E3F6
:100C30006CD00895E8E9FCE00FA10055102F110FCA
:100C4000110F000F010FE00FFF1D95FF0AC09F7DE0
:100C500005911591F80109950DAD03950DAF30DBA8
:100C60001AC093FF18C0329605911591FF93EF9328
:100C7000F8010DAD002309F009950FA103950A3580
:100C80000CF00FE458D0EF91FF91A591B5910A2F88
:100C90000B2B09F046D00895C201000044015718FB
:100CA0006A064C01F00604075401BE06D4065C0136
:100CB0000C072007640126073A076C014207560714
:100CC0007401A506B7067C015E07760784017E07DE
:100CD000960700000895ED91FD9112970FEFBAD994
:100CE0000895F9DFA8A7B9A70895F5DFAAA7BBA7BC
:100CF0000895A8A5B9A5D4D9F8A6F9A60895AAA5D6
:100D0000BBA5CED9FAA6FBA60895977F0EA3F1DF67
:100D1000D7DA0895A8A5B9A51DDAAAA5BBA51ADA40
:100D20000895D9DFACA7BDA70895ACA5BDA5B8D9D6
:100D3000FCA6FDA60895977F0FA3FDAEC1DAF5DFEF
:100D40000895ACA5BDA506DA08950AAD01950395F1
:100D50000AAF01D008950AADEAE6FDE06BDEE4E7F4
:100D6000F1E000831183EDDF0895C311D8110AADBE
:100D70001E8D19F00CD509E50FA308950EA9039552
:100D800007310CF004E10EAB01D008950EA9045117
:100D9000E2EAFDE04FDEE4E5F1E000831183D1DF1C
:100DA000089571108E10AD100EA910910002011758
:100DB000B1F0163169F48CD40EA91F85112321F0EE
:100DC000053159F0ACD409C0043139F0A8D405C0BC
:100DD000063111F47DD401C0A2D409E50FA3089512
:100DE0000DA9019503950DAB01D008950DA9002320
:100DF00019F40EE410E202C002E310E2ECE4F1E0C8
:100E0000008311839EDF08950DA91B85011719F03A
:100E1000E8D309E50FA308950FA9019503950FAB3A
:100E200001D008950FA9002319F404EE11E202C0C5
:100E300006E112E2ECE5F1E00083118382DF089520
:100E40000E851FA9011709F026D4089508AD019554
:100E5000039508AF01D0089508AD002319F000E80C
:100E600012E202C004E612E2E4E6F1E0008311833C
:100E700068DF089508AD1D85011719F040D409E514
:100E80000FA3089509AD0195039509AF01D0089509
:100E900009AD002319F008E213E202C00CE013E2EE
:100EA000ECE6F1E0008311834CDF089509AD1B8D62
:100EB000011719F049D409E50FA308950E850E1105
:100EC00008950BAD019503950BAF01D008950BADBF
:100ED000002319F006E614E202C008E214E2ECE78F
:100EE000F1E0008311832DDF089508950BAD1C8D73
:100EF000011719F0A7D309E50FA308950E850E1168
:100F000008950CAD019503950CAF01D008950CAD7B
:100F1000002319F004E115E202C006ED14E2E4E852
:100F2000F1E0008311830DDF089508950CAD1D8D50
:100F3000011719F09FD309E50FA308950B850DAB99
:100F400055DF0C85002311F016E105C014E10F8573
:100F5000002309F015E11EAB1093000217DF0E8588
:100F60000FAB60DF0D8508AF77DF0B8D09AF90DF2A
:100F70000E8D0AAFF0DE0C8D0BAFA9DF0D8D0CAF1F
:100F8000C6DF0895569A5E9808950D8500FF4E9A23
:100F900008955E98089557985F9A089508A90F3F9D
:100FA00071F4E8AAA9A9BAA90A2F0B2B41F4A8E168
:100FB000B1E0E2EAFDE100EF4DD8A9ABBAAB08958C
:100FC0000FEF08ABA9A9BAA96BD8F9AAFAAAFF82B0
:100FD000089508850F8308950C8D00FD0895AEA532
:100FE000BFA50A2F0B2B41F4A8E1B1E0ECEBFDE12A
:100FF0000FEF30D8AEA7BFA70895AEA5BFA550D8B4
:10100000FEA6FFA627D0089509890F3F71F0FF9330
:10101000EF93E4E2FCE203950770098B000FE00F09
:10102000FF1D85909490EF91FF910895ABA9BCA905
:101030000A2F0B2B41F4A0E0B1E0E8E4FBE100E56E
:1010400009D8ABABBCAB0895ABA9BCA929D8FBAA06
:10105000FCAA08950BA106FD0EC00E85002329F4FD
:10106000F0921801F092190106C0E6E9FDE1E09363
:101070001801F09319010895A7E0B0E016C0A0E0B0
:10108000B0E013C0A6E0B0E010C0A3E0B0E00DC037
:10109000A2E0B0E00AC0A4E0B0E007C0A1E0B0E088
:1010A00004C0A5E0B0E001E000C00090050200200F
:1010B00019F400BD16E089D30895A7E0B0E012C08E
:1010C000A0E0B0E00FC0A6E0B0E00CC0A3E0B0E04C
:1010D00009C0A4E0B0E006C0A2E0B0E009C0A1E011
:1010E000B0E000C011E071D30F3F09F4002708956C
:1010F00011E06BD30F3F09F40E2D08950F93098172
:101100008EE1080F0C330CF00C5361D4882329F4C2
:1011100065DA8981081729F0F8CF17D495D30F9194
:10112000089588E50F9108958F9355D4882311F47D
:1011300055DAFBCF8F9100D408954DD4882311F454
:101140004DDAFBCF1DD408958F9345D4882311F435
:1011500045DAFBCF8F9118D008953DD4882311F440
:101160003DDAFBCF1DD408950F9335D4882311F4B5
:1011700035DAFBCF0F91002319F0E8E1FEE200C45D
:10118000ECE1FEE2FDC30895E4E1FEE2F9C3A3D879
:1011900095FF02C09F7DF6D821DAABD80023C1F7B6
:1011A0000895F5DFF4DF0895C8DFCEDFF0DF08959E
:1011B000C4DFCADFF6DF08958F931F930F932F9339
:1011C0003F93BF93AF93FF93EF930F921F92BDD3C3
:1011D0003BD3883509F08FC0EAE5FCE2AEDF8EDF55
:1011E000A3DFB2DF843509F43AC0843409F46BC05C
:1011F000833509F466C08C3411F481D27CC081340B
:1012000011F449D278C0863511F4B7D274C0833452
:1012100011F4E7D170C08E3411F45AD26CC080350D
:1012200011F47DD268C0823411F48ED264C081354D
:1012300011F408D260C0823511F41CD25CC086342F
:1012400011F4A5D258C0883411F4C9D254C08D34D9
:1012500019F40E942F1B4FC0883579F1BDCFE4E807
:10126000FCE26BDF56D040F175D159DC6DDFECE963
:10127000FCE263DF4ED000F165D166DFE4EBFCE217
:101280005CDF47D0C8F00E85002351F48F9389812D
:101290008F9387DA8F9110D109810817C9F38F9145
:1012A00047D1EA8E09810A9509830DDB9B7791DE90
:1012B0004BDF002761D004C07BDBE6EDFDE23DDFC4
:1012C0001AC074D118C0ECECFCE237DF22D0A8F3CE
:1012D00059D13ADFE4EEFCE230DF1BD070F34AD1A3
:1012E00033DFECEFFCE229DF14D038F33BD12CDF05
:1012F000002742D000C028DFEA8E1F900F90AF91E8
:10130000BF91EF91FF913F912F910F911F918F917D
:101310000895F4DE09DF883511F4089408950DD09E
:10132000C0F3082FEBDE00DF8835B9F306D0D0F329
:101330001AE0019F800D88940895803328F08A3345
:1013400018F480538894089508940895E4E3FCE227
:10135000F4DE82E3E9DE8EE2E7DE87E3E5DEF4DE5B
:1013600008955CD28F9382958F7064D28D938F9104
:101370008F7060D28D93089500900402002019F0C0
:10138000F09204027DD027D3882311F427D9FBCF14
:10139000FF93EF93BF93AF930F93A6E0B2E011D00A
:1013A00080E28D9329D00F91002321F08DE08D9361
:1013B0008AE08D93FD92F4D2AF91BF91EF91FF91AE
:1013C00008958C81CEDF8DE28D938D81E0E2FEE287
:1013D0008A95880F880FE80FFF1D85918D93859161
:1013E0008D9385918D938DE28D9382E38D9380E330
:1013F0008D938E81B6DF08958B81B3DF8AE38D9361
:101400008A81AFDF8AE38D938981ABDF0895E3D2D0
:10141000882311F4E3D8B0CFFF93EF93BF93AF933A
:101420000F93A6E0B2E0E8DF0F91002321F08DE0FA
:101430008D938AE08D93FD92B3D2AF91BF91EF91DE
:10144000FF910895098103950C3308F00027098363
:101450000E946001AEDA08950A8103950C3308F00A
:1014600000270A830E946001A4DA08950B81039586
:10147000083108F000270B830E9460019ADA089572
:101480000F938F9315E0E6D28F73B8D180320CF0B2
:101490008E2D8C8317E0DED28F71B0D18D300CF0A1
:1014A0008E2D8D8318E0D6D2A9D183360CF08827F3
:1014B0008E838F910F9108958F9312E0CBD28F7707
:1014C0009DD18C330CF0882789838F9108958F9359
:1014D00012E0C0D287FD62DD8F7790D18C330CF0A3
:1014E0008827898313E0B6D28F7788D18C330CF0AC
:1014F00088278A8314E0AED28F7380D188310CF0B4
:1015000088278B838F91089580910502882379F431
:10151000898184D112E0082FBFD28A817FD113E064
:10152000082FBAD28B817AD114E0082FB5D2089552
:101530008F93082F0C3320F4898370D112E0ACD242
:101540008F910895082F0C3320F48A8367D113E01C
:10155000A3D20895082F083120F48B835FD114E0C3
:101560009BD20895082F003220F48C8357D115E0C8
:1015700093D20895082F0D3020F48D834FD117E0BA
:101580008BD20895082F8E8349D118E085D2089513
:101590008827CEDF8827D6DF8827DCDF81E0E2DFFF
:1015A00081E0E8DF8827EEDF7CDD0895CFDE0027CD
:1015B000E3DE80E2B9DD82E50E85002309F081E4F7
:1015C000B3DD0D85002311F48CE4AEDD0B8D00231B
:1015D00011F482E4A9DD098D002311F086E5A4DD74
:1015E00008952F93E4E1FDE2A8DD0B85002339F097
:1015F0001FD2002722271A85E8E4FBE109C015D095
:1016000013D20E2D2FEF8824992411E0E0E4F5E2A7
:101610001987E0930001F09301011B8D112309F458
:10162000298B0B87A1DD2F9108950C8D002321F0CC
:101630001EE318871F83FC8E0D8D002309F0FD8E9D
:10164000AFD908950E8500FD04C0E4E9FDE275DD23
:1016500010C0EAE7FDE271DD0C8D002319F01EE3F6
:10166000002702C012E00E2D18871F830C8F7CDD2F
:1016700097D908950E8500FD04C0E4E9FDE25DDD23
:1016800009C0E6E8FDE259DD0D8D019503950D8F4A
:101690006BDD86D90895E4E5FDE24FDD0E8500237C
:1016A00039F0C3DF0027F0921801F092190107C04A
:1016B0000395E6E9FDE1E0931801F09319010E8727
:1016C000E7DC52DD0091050200FF0E94C20108958F
:1016D0000B85002399F4EAE2FDE22FDD0C8500235F
:1016E00019F000271FE002C0039517E00C87198747
:1016F0001A87CBDC0195039537DD11DA0895ECE309
:10170000FDE21BDD0D85002311F0002702C00395CB
:1017100040DC0D87B4DC0195039526DD0895ECE4EB
:10172000FDE20BDD0F85019503950F87B4DC1EE309
:1017300000FD1AE40195039517DD2F2D03D0D5D9AF
:1017400075D9089573D90895E6E6FDE2F6DC0B8DB0
:10175000019503950B8F0F9395DC0195039504DD9F
:101760000F911B85112341F4002329F00FEF098B02
:101770008824992401C0F98A0895E2E4FDE2DDDCC1
:10178000098D01950395098F89DCEEDC0895E2EC63
:10179000FDE2D3DC0E8D002331F00027E091010241
:1017A000F091020203C00395E0E0F0E0E093040151
:1017B000F09305010E8F60DC01950395D5DC08954B
:1017C000A5E0B0E011E001D00895A1BDB2BD119631
:1017D00011FDFA9A1FBBF999FECF00B50895E0E517
:1017E000FEE2ABDC0895222738E0000F221F21170C
:1017F00010F00395211B3A95C1F708950F921F929F
:101800000F938F9382958F700AE0809F002D8F91A8
:101810008F70800F0F911F900F900895082F1AE07E
:10182000E2DF07700295022B802F08951AE0DBDFBC
:1018300007700895FF93EF93ECEFFBE2E80FFF1DB5
:101840008491EF91FF910895813624F08B3710F445
:1018500000E2801B089510E41093C400F092C500CC
:10186000F092C00018E41093C10016E01093C2007B
:10187000EB8AFF8AF88EFC8AFD8A1FEF1E8B089583
:101880001091C10010691093C10008950F930FB714
:101890000F931F93FF93EF930E890F3F79F00395FA
:1018A000E6E0F2E0E00FFF1D1081112319F40FEFC5
:1018B000EB8A02C01093C6000E8B12C0EC89FD8922
:1018C0000E2F0F2B39F0EF5FFF4F1491112321F4EE
:1018D000FC8AFD8AEB8A04C01093C600EC8BFD8B5A
:1018E000EF91FF911F910F910FBF0F9118950F93DB
:1018F0000FB70F930BA102FD0C948E1B1F932F9318
:101900003F93FF93EF932091C6000F89302F0395EB
:101910000F70188D011739F00F8BE6E8F2E0E30F36
:10192000FF1D20839160EF91FF913F912F911F91B7
:101930000F910FBF0F9118950F930B890023E9F3B7
:10194000FB8A8093C6000F91089590FFFECF0F93FE
:101950001F93FF93EF931F89088D8827011751F07C
:10196000E6E8F2E0E00FFF1D808103950F70088F1D
:10197000011709F49E7FEF91FF911F910F91089538
:101980000F93FF93EF930B890023E9F3FB8AEC8B12
:10199000FD8B04910093C600EF91FF910F91089584
:1019A0000F93FF93EF930B890023E9F3FB8AFE8AE1
:1019B000E6E0F2E00081002321F40FEF0E8BEB8ACA
:1019C00002C00093C600EF91FF910F910895882700
:1019D00090FD839508958B8908951F930F9328D0C8
:1019E0001FE000E459D01EE001E856D011E001E10B
:1019F00053D00F911F9108951FE000E44DD011E0E6
:101A000001E14AD008951EE000E846D011E000E16F
:101A100043D008951FE000E43FD01EE001E83CD031
:101A200011E001E139D008951DE000E835D00895B6
:101A30001DE0002731D008950000000000000000E4
:101A4000000000000000000008953C9A3D9A449A6E
:101A5000459A08953F9333273A9519F4E09203028B
:101A600017C0B1F067D0E8DF02EA3FD0E5DF33D03E
:101A700098F3012F3AD0E0DF2ED070F355D05AD032
:101A800003EA33D0D9DF27D038F33CD0449A459AC3
:101A90004BD0802F3F9108953F9333273A9519F407
:101AA000E092030215C046D0C7DF0F9302EA1DD0B3
:101AB000C3DF11D00F9190F30F93012F16D00BD0ED
:101AC0000F9160F30F9311D006D00F9138F30000FF
:101AD0002BD03F9108953C98449A0894459AACDFE6
:101AE000349B889445983C9A08953F9338E0449AF3
:101AF000000F08F04498459A9FDF45983A95B9F74A
:101B00003F9108953F933C98449A00E038E0459A0D
:101B1000089492DF349B8894001F45988DDF3A9596
:101B2000B1F73C9A3F9108954498459A000000000F
:101B3000449A0895449A459A000000004498000091
:101B400000004598000008957AEB7AD90080E88378
:101B5000EB89EB8CE88CE580D98CD900862483272F
:101B60007D277A247A187D1583158618861B831E97
:101B70007D1E7A1B00E086E389E989EC86EC83E927
:101B800080EC7DEC7AE977E377E07A00E380E98026
:101B9000001F831C801C8016801383138616891CEB
:101BA000891F861F7A1C771677137A0080FE80F2D1
:101BB000008DFE8CF9009AFC99F700A6F8A5F400B8
:101BC000B3F4B1EF00BFEEBAE500CAE6C7E200D455
:101BD000DED0DA00DDD5D9D100E5CBE1C800EDBF1C
:101BE000E4BA00F3B4EEB200F7A7F3A600FB9BF64D
:101BF0009A00FD8EF88D00FD80F18000FD73F87471
:101C000000FB66F66700F75AF35B00F34DEE4F00FA
:101C1000ED41E44600E536E13900DD2CD93000D451
:101C200023D02700CA1BC71F00BF13BA1C00B30D67
:101C3000B11200A609A50D009A05990A008D038C22
:101C400008007F037F0F0072037308006505660AB2
:101C50000059095A0D004C0D4E12004113461C004C
:101C6000351B381F002B232F2700222C2630001A6B
:101C7000361E390012421B47000C4D114F00085A06
:101C80000C5B000466096700027307740002810E92
:101C90008100028E078D00049B099A0008A70CA6FC
:101CA000000CB411B20012BF1BBA001ACB1EC80040
:101CB00022D526D1002BDE2FDA0035E638E20040AF
:101CC000EE45E5004CF44EEF0059F85AF40065FC7F
:101CD00066F70072FE73F9FFB5E4B5D20000D2BB1F
:101CE000D5BEDBBEDEBBDEB8D2ACDEAC0000E04C65
:101CF000D44CDD55DD430000B831AC31AC28B528FB
:101D0000B825B822B51FAF1FAC22000047315331B0
:101D1000532E502B4D254D1F0000224C1F4F1F529C
:101D2000225528552B522B4F284C224C1F491F4619
:101D3000224328432B462B49284C000021BE21ACCE
:101D4000000027BB2ABE30BE33BB33AF30AC2AAC59
:101D500027AF27BB000049E449D2000053E453D227
:101D6000FF00B2A4B2A6BAA6BA9AB29AB29C00BEBA
:101D70009ABE9EC49EC49ABE9A00C49AC4A600C7C6
:101D80009AC7A6CDA6CFA4CFA2CDA0C7A000CDA0B4
:101D9000CF9ECF9AFF007CBA80C684BA0082BE7EF6
:101DA000BEFF7CBA7CC682C684C484C282C07CC0AA
:101DB00082C084BE84BC82BA7CBAFF007CBA7CC676
:101DC00082C684C484C282C07CC0FF00A999AC9939
:101DD000AD98AD94AC93A993A99900B999B599B56B
:101DE00093B99300B896B59600C093C099C297C4B2
:101DF00099C49300CB98CC99CE99CF98CF94CE9399
:101E0000CC93CB94CB98FF003A933A993D993E9866
:101E10003E973D963A960046994694479349934A91
:101E200094004A994A93005698559953995298525A
:101E300097539655965695569455935393529400AE
:101E40005E995E93005E9662960062936299007658
:101E5000997A9900789978930082988399859986E0
:101E60009886948593839382948298009E989D99F6
:101E70009B999A989A979B969D969E959E949D93D2
:101E80009B939A9400A699AA9900A899A89300B246
:101E900093B499B69300B595B39500BE93BE99C11E
:101EA00099C298C297C196BE9600C196C295C29338
:101EB00000CA99CE9900CC99CC93FF0029EC2FEC65
:101EC00031EA31E22FE029E029EC0035EC35E23748
:101ED000E03BE03DE2003DEC3DE00041EC49EC0040
:101EE00045EC45E00055EA53EC4FEC4DEA4DE24F2E
:101EF000E053E055E20059EC59E00059E661E60094
:101F000061E061EC0065EC6DEC0069EC69E000718A
:101F1000E071EC77EC79EA79E877E671E60077E64C
:101F200079E479E0007DEA7FEC83EC85EA85E28361
:101F3000E07FE07DE27DEA0089E089EC91E091ECD0
:101F40000097E09BE00099E099EC0097EC9BEC0097
:101F5000A1ECA9E000A9ECA1E000B9ECBDE0C1EC66
:101F600000C5EAC7ECCBECCDEACDE8C5E0CDE0009A
:101F7000D3E0D3E4D7E4D7E0D3E000DDECE5ECE553
:101F8000EAE3E8E1E4E1E0FF29C229CE2FCE31CC3B
:101F900031CA2FC829C82FC831C631C42FC229C29F
:101FA0000035CC37CE3BCE3DCC3DC43BC237C235ED
:101FB000C435CC0041CC43CE47CE49CC49C447C2FE
:101FC00043C241C441CC004DCE55CE0051CE51C28A
:101FD000FF0029BA2FBA31B831B02FAE29AE29BAD5
:101FE000003DBA35BA35AE3DAE003BB435B4004124
:101FF000AE41BA45B649BA49AE004DB84FBA53BA28
:1020000055B855B053AE4FAE4DB04DB8FF0031A4EA
:102010002FA62BA629A4299C2B9A2F9A319C0035F8
:102020009A39A63D9A003B9E379E0041A6419A49A7
:102030009AFF59A45BA65FA661A4619C5F9A5B9A14
:10204000599C59A400659A65A66D9A6DA6FF59A47E
:102050005BA65FA661A4619C5F9A5B9A599C59A498
:10206000006DA665A6659A0065A06BA00079A671B3
:10207000A6719A0071A077A0FF0029862992318667
:102080003192003592358837863B863D88003D92F7
:102090003D860041864192458E499249860055927F
:1020A0004D924D86558600538C4D8C005986599221
:1020B0005F926190618E5F8C598C005F8C618A6148
:1020C000860067866B8600698669920067926B92CC
:1020D0000079907792739271907188738677867980
:1020E00088FF8D928D8600959097929B929D909DF2
:1020F0008E95869D8600A192A18600A18CA98C0058
:10210000A986A99200AD86AD92B392B590B58EB373
:102110008CAD8C00B38CB58AB586FF0089908B920C
:102120008F929190918E89869186009D8C958C9B43
:10213000929B8600A192A18600A18CA98C00A98601
:10214000A99200AD86AD92B392B590B58EB38CAD29
:102150008C00B38CB58AB586FF0089908B928F92E4
:10216000919091888F868B8689888990009D929521
:1021700092958600958C9B8C00A992A192A18600D5
:10218000A18CA78CFF002972297E2D7A317E3172B5
:10219000003572397E3D72003B76377600497C47C8
:1021A0007E437E417C417A4378477849764974473B
:1021B0007243724174004D7E557E00517E51720013
:1021C000617E597E59726172005F7859780065723C
:1021D000657E6B7E6D7C6D7A6B786578006B786D53
:1021E000766D72FF7D727D7E837E857C857A8378B5
:1021F0007D780083788576857200897E917E008D5A
:102200007E8D72009D7C9B7E977E957C95749772E7
:102210009B729D74FF007D72817E85720083767F44
:102220007600897E8D72917E009572957E9B7E9D53
:102230007C9D7A9B789578009B789D769D72FF00B7
:10224000296A295E315E003D6A356A355E3D5E0071
:102250003B64356400416A476A49684960475E41AA
:102260005E416AFF59685B6A5F6A616861605F5ED0
:102270005B5E5960596800655E656A6D5E6D6AFFF8
:1022800059685B6A5F6A616861605F5E5B5E596046
:102290005968006D6A656A655E0065646B64007903
:1022A0006A716A715E0071647764FF00294A295679
:1022B0002F56315431522F5029502F50314E314C1E
:1022C0002F4A294A003556354C374A3B4A3D4C0087
:1022D0003D563D4A00414A415647564954495247A6
:1022E000504150004750494E494A004D4A4D5655BD
:1022F0004A5556005B4A5F4A005D4A5D56005B5690
:102300005F5600654A65566D4A6D56FF7D547F568F
:1023100083568554854C834A7F4A7D4C7D54008981
:102320004A8956914A9156FF7D547F56835685546B
:10233000854C834A7F4A7D4C7D540091568956894D
:102340004A0089508F50009D569556954A009550E9
:102350009B50FF0029422F42314031382F36293619
:1023600029420037363B3600393639420037423B86
:10237000420041364542493600473A433A004D4211
:102380004D365536FF006D426542653600653C6B43
:102390003C0071427138733677367938007942796A
:1023A00036007D427D36853600894289369136FF7A
:1023B00065366542693E6D426D360073367736008C
:1023C000753675420073427742007D367D42853610
:1023D0008542FF00312C2F2E2B2E292C292A2B2829
:1023E0002F28312631242F222B2229240035223573
:1023F0002E3B2E3D2C3D2A3B28352800492E412ED0
:1024000041224922004728412800552E4D2E4D22B9
:1024100055220053284D2800592E5F2E612C61242F
:102420005F225922592EFF007122712E7922792EB6
:10243000007D2C7F2E832E852C852483227F227D78
:10244000247D2C008922892E8F2E912C912A8F2871
:102450008928008F2891269122009522952E992A6D
:102460009D2E9D22FF00792E712E712200712877FA
:1024700028007D22812E85220083267F2600912C34
:102480008F2E8B2E892C892A8B288F289126912498
:102490008F228B22892400952E9D2E00992E992221
:1024A000FF00291A2F1A311831102F0E290E291A60
:1024B00000370E3B0E00390E391A00371A3B1A004E
:1024C000410E411A471A491849164714411400474A
:1024D000144912490EFF590E591A610E611A00650E
:1024E00018671A6B1A6D186D106B0E670E65106504
:1024F0001800710E711A771A7918791677147114F9
:102500000077147912790E007D0E7D1A8116851AD6
:10251000850EFF00590E591A5F1A611861165F1473
:102520005914005F146112610E006D1A651A650E70
:102530006D0E006B14651400711A750E791AFF0088
:1025400001FE0101FE01FEFE01FEFE010101FEFE93
:1025500001FE0101FE01FEFEFF0080EC8080FF8B8A
:10256000EC8080FF96EA8080FFA1E78080FFABE3EC
:102570008080FFB6DE8080FFBFD88080FFC8D1801A
:1025800080FFD0C98080FFD7C08080FFDDB680800B
:10259000FFE2AC8080FFE6A28080FFE9978080FFA9
:1025A000EB8C8080FFEB808080FFEB758080FFE903
:1025B0006A8080FFE65F8080FFE2558080FFDD4A11
:1025C0008080FFD7418080FFD0388080FFC8308076
:1025D00080FFBF298080FFB6238080FFAB1E8080F4
:1025E000FFA11A8080FF96178080FF8B158080FFE7
:1025F00080158080FF74158080FF69178080FF5EE2
:102600001A8080FF541E8080FF4A238080FF40296B
:102610008080FF37308080FF2F388080FF28418006
:1026200080FF224B8080FF1D558080FF195F8080D6
:10263000FF166A8080FF14758080FF14808080FF01
:10264000148C8080FF16978080FF19A28080FF1D68
:10265000AC8080FF22B68080FF28C08080FF2FC919
:102660008080FF37D18080FF40D88080FF49DE80A6
:1026700080FF54E38080FF5EE78080FF69EA80800E
:10268000FF74EC8080FF828080E67E808280FF8104
:10269000808AE67E818180FF818095E47E818180D1
:1026A000FF81809FE27E818180FF8180A9DE7E8123
:1026B0008180FF817FB3D97E82817FFF817FBBD301
:1026C0007E82817FFF817FC4CC7E82817FFF817F7C
:1026D000CBC57E82817FFF817FD2BC7E82817FFFDE
:1026E000807FD8B37F82807FFF807FDDAA7F82805A
:1026F0007FFF807FE1A07F82807FFF807FE3967FE6
:1027000082807FFF807FE58B7F82807FFF7F7EE5F9
:102710008080827F7EFF7F7FE57680827F7FFF7F64
:102720007FE36B80827F7FFF7F7FE16180827F7F9D
:10273000FF7F7FDD5780827F7FFF7E7FD84D818244
:102740007E7FFF7E7FD24581827E7FFF7E7FCB3C76
:1027500081827E7FFF7E7FC43581827E7FFF7E7F88
:10276000BB2E81827E7FFF7E7FB32881827E7FFFAA
:102770007E80A92381817E80FF7E809F1F81817E54
:1027800080FF7E80951D81817E80FF7E808A1B81F7
:10279000817E80FF7E817F1B82807E81FF7E8175AE
:1027A0001B81807E81FF7E816A1D81807E81FF7E0C
:1027B00081601F81807E81FF7E81562381807E81A2
:1027C000FF7E814D2881807E81FF7E82442E817F25
:1027D0007E82FF7E823B35817F7E82FF7E82343C1B
:1027E000817F7E82FF7E822D45817F7E82FF7F8278
:1027F000274E807F7F82FF7F822257807F7F82FFEC
:102800007F821E61807F7F82FF7F821C6B807F7F43
:1028100082FF7F821A76807F7F82FF80821A817F8B
:102820007E8082FF80821A8B7F7F8082FF80821C65
:10283000967F7F8082FF80821EA07F7F8082FF80C4
:102840008222AA7F7F8082FF808227B37F7F80825F
:10285000FF81822DBC7E7F8182FF818234C57E7F95
:102860008182FF81823BCC7E7F8182FF818244D343
:102870007E7F8182FF81824CD97E7F8182FF818130
:1028800056DE7E808181FF818160E27E808181FFD2
:1028900081816AE47E808181FF818175E67E80810D
:1028A00081FF828080BC7E808280FF818086BC7EAA
:1028B000818180FF81808CBB7E818180FF818092BD
:1028C000BA7E818180FF818098B77E818180FF817F
:1028D0007F9EB47E82817FFF817FA3B17E82817FD4
:1028E000FF817FA8AD7E82817FFF817FACA97E8240
:1028F000817FFF817FB0A47E82817FFF807FB39E36
:102900007F82807FFF807FB6997F82807FFF807F7C
:10291000B9937F82807FFF807FBA8D7F82807FFF27
:10292000807FBB877F82807FFF7F7EBB8080827FAE
:102930007EFF7F7FBB7A80827F7FFF7F7FBA74803C
:10294000827F7FFF7F7FB96E80827F7FFF7F7FB630
:102950006880827F7FFF7E7FB36281827E7FFF7E81
:102960007FB05D81827E7FFF7E7FAC5881827E7FDB
:10297000FF7E7FA85481827E7FFF7E7FA35081826D
:102980007E7FFF7E7F9E4D81827E7FFF7E80984A84
:1029900081817E80FF7E80924781817E80FF7E8064
:1029A0008C4681817E80FF7E80864581817E80FF8E
:1029B0007E817F4582807E81FF7E81794581807E18
:1029C00081FF7E81734681807E81FF7E816D47819C
:1029D000807E81FF7E81674A81807E81FF7E816269
:1029E0004D81807E81FF7E825C50817F7E82FF7E72
:1029F000825754817F7E82FF7E825358817F7E8200
:102A0000FF7E824F5D817F7E82FF7F824C63807F6D
:102A10007F82FF7F824968807F7F82FF7F82466E50
:102A2000807F7F82FF7F824574807F7F82FF7F82ED
:102A3000447A807F7F82FF808244817F7E8082FF14
:102A4000808244877F7F8082FF8082458D7F7F8068
:102A500082FF808246937F7F8082FF808249997FB8
:102A60007F8082FF80824C9E7F7F8082FF81824FA9
:102A7000A47E7F8182FF818253A97E7F8182FF8134
:102A80008257AD7E7F8182FF81825CB17E7F8182B1
:102A9000FF818261B47E7F8182FF818167B77E8002
:102AA0008181FF81816DBA7E808181FF818173BBCD
:102AB0007E808181FF818179BC7E808181FF24536A
:102AC000245526552653245300244F244D264D26A5
:102AD0004F244F00445344554655465344530044F5
:102AE0004F444D464D464F444FFF644B68576C4B27
:102AF000006A4F664F00704B705774537857784B8D
:102B0000FF00644B64576A576C556C536A516451AB
:102B10000000704B705774537857784BFF0099152D
:102B2000A315A615AE15BC15C115CB15D815DF1507
:102B3000F015040C060E0A0E0C0C0C040A02060218
:102B40000404040CFF00080E0802FF00040C060E2B
:102B50000A0E0C0C0C0A04020C02FF00040C060EF8
:102B60000A0E0C0C0C0A0A080C060C040A020602D7
:102B700004040006080A08FF0C0804080A0E0A02EA
:102B8000FF000C0E040E04080A080C060C040A02CE
:102B900006020404FF000C0C0A0E060E040C0404CA
:102BA00006020A020C040C060A0806080406FF00C6
:102BB000040E0C0E0C0C0A0A08060802FF00060898
:102BC000040A040C060E0A0E0C0C0C0A0A0806086D
:102BD0000406040406020A020C040C060A08FF009C
:102BE0000C0A0A080A080608040A040C060E0A0E53
:102BF0000C0C0C040A0206020404FF0030313233CC
:102C00003435363738394142434445460C010203D6
:102C10000405060708090A0B0C0102030405060750
:102C200008090A0B0000010001010001FF01FF007B
:102C3000FFFF00FF447574636874726F6E697820DB
:102C4000415652204F7363696C6C6F73636F70658C
:102C500020436C6F636B20560000456E74657220D4
:102C6000636F6D6D616E642028412C422C432C44AF
:102C70002C462C482C4C2C4E2C502C532C542C567F
:102C8000293A0000456E74657220322064696769D4
:102C90007420686F7572733A20202000456E746549
:102CA000722032206469676974206D696E7574657D
:102CB000733A2000456E746572203220646967693A
:102CC00074207365636F6E64733A2000456E74659B
:102CD00072203220646967697420796561723A20D4
:102CE00020202000456E7465722032206469676977
:102CF00074206D6F6E74683A20202000456E7465F4
:102D0000722032206469676974206461793A2020F6
:102D10002020200043616C6962726174696F6E20CB
:102D20005061747465726E2000004E756D65726935
:102D30006320646973706C61792000004C45442005
:102D40000000566572626F7365200000414D2F5080
:102D50004D20000041565220436C6F636B204D6143
:102D60007374657220004275726E2D696E20507208
:102D70006576656E74696F6E200046617374204DD0
:102D80006F646520000052657665727365204D6F33
:102D900064652000526571756573746564206D6F9C
:102DA00064652072657175697265732041565220A1
:102DB000636C6F636B204D6173746572204D6F643B
:102DC0006500416C6C2044696769747320646973A1
:102DD000706C6179200043616E63656C206F7220B6
:102DE00054696D656F7574004E6F7420456E74651F
:102DF00072696E672044656D6F204D6F64650000D9
:102E0000505053207369676E616C2069676E6F72F2
:102E1000656400000D0A00004F6E00004F666600FA
:102E20004A616E1F4665621C4D61721F4170721EC1
:102E30004D61791F4A756E1E4A756C1F4175671F7B
:102E40005365701E4F63741F4E6F761E4465631F7B
:102E5000447574636874726F6E6978204F73636928
:102E60006C6C6F73636F706520436C6F636B20488D
:102E7000656C703A0D0A413A20546F67676C6520A3
:102E80004D617374657220436C6F636B206265746F
:102E90007765656E2041565220616E64205254431E
:102EA0000D0A423A20546F67676C65204275726E56
:102EB0002D696E2070726576656E74696F6E0D0A8D
:102EC000433A20446973706C61792043616C696294
:102ED000726174696F6E207061747465726E0D0A30
:102EE000443A204368616E676520446174650D0A49
:102EF000463A20546F67676C6520416C6C204469CA
:102F00006769747320446973706C61790D0A4C3A77
:102F100020546F67676C65204C454420626C696E75
:102F20006B696E670D0A4E3A20546F67676C6520B7
:102F30004E756D6572696320446973706C617920A8
:102F40000D0A503A20546F67676C6520414D2F5031
:102F50004D200D0A533A20446973706C61792053F7
:102F60007461747573200D0A543A204368616E676A
:102F7000652054696D650D0A563A20546F67676C79
:102F80006520566572626F7365204F757470757435
:102F90000D0A0000ECECFDE1E0931401F093150143
:102FA0000895E0E0F0E0E0931401F0931501089536
:102FB0000C850023D9F50E94680B36C00C850023D0
:102FC000A9F10E94680B30C00F85002379F50E949B
:102FD0008F0B2AC00F85002349F10E948F0B24C05C
:102FE0000E8D002319F50E94C70B1EC00E8D002305
:102FF000E9F00E94C70B18C00D850023B9F40E94A8
:103000007F0B12C00D85002389F00E947F0B0CC03E
:103010000B85002361F00E94F10A06C00B85002396
:1030200031F40E94F10A00C00E94A40800C0089573
:10303000098D0023E1F30E94BD0BF6CF098D00231B
:10304000B1F70E94BD0BF0CF0E85002381F30E94E3
:103050004B0BEACF0E85002351F70E944B0BE4CFB8
:103060000C8D002321F30E94220BDECF0C8D002358
:10307000F1F60E94220BD8CF0D8D0023C1F20E94E1
:103080003A0BD2CF0D8D002391F60E943A0BCCCF94
:103090000895F98A08950E94FD0708950E94EC079B
:1030A00008950E94E00708950E94CE07089501E068
:1030B000009305020E94CA17D3DFDEDFA9DFE6EF27
:1030C000F2E0EEAFFFAFE8E6F2E30E94D408ECE0F6
:1030D000F3E30E94D4080E94D8170E94F017EAE395
:1030E000F3E30E94D4080E94F617ECE5F3E30E9494
:1030F000D4080E94E4170E94DE17EAE7F3E30E9477
:10310000D4080E94EA17ECE9F3E30E94D408EEEB3E
:10311000F3E30E94D4080E94E4170E94C7080E94AB
:10312000F0170E94C7080E94EA170E94C7080E9471
:10313000F6170E94D8170E94C7080E94F6170E942F
:10314000DE170E94C7080E94F0170E94D8170E943D
:10315000C7080E94F6170E94EA170E94DE170E9415
:10316000C7080E94FC17EAEDF3E30E94D8080E940A
:103170000218E4EFF3E30E94D8080E940E18E8E07A
:10318000F4E30E94D8080E940818E2E2F4E30E94E7
:10319000D8080E942A18E4E3F4E30E94D8080E94A9
:1031A0003618E6E6F4E30E94D8080E94D1080E948F
:1031B0003018E8E7F4E30E94D8080E944218ECE8CF
:1031C000F4E30E94D8080E943618EEE9F4E30E9466
:1031D000D8080E94D1080E94150B009305020E9496
:1031E0005418ECEDF4E30E94D8080E94D10803E0E3
:1031F000009305020E9451180E944E18EEE2F5E37A
:103200000E94D8080E94D1080E944B180E941608FC
:10321000EEE7F5E30E94D80805E0009305020E945E
:1032200024080E944918ECE9F5E30E94D8080E949E
:10323000D108F09205020E944818ECE1F3E0EEAFED
:10324000FFAFE8EEF2E30E94D8080E94D108E6EF53
:10325000F2E0EEAFFFAFECEFF5E30E94D4080E947E
:10326000D1170E94C2010895546869732064656D86
:103270006F206D6F64652073686F777320736F6D57
:1032800065206F6620746865206361706162696C97
:103290006974696573206F6620746865204475746D
:1032A000636874726F6E69780D0A415652204F73CD
:1032B00063696C6C6F73636F706520436C6F636BD5
:1032C0002E20497420707265736572766573207460
:1032D0006865207374617465206F6620796F7572FC
:1032E00020636C6F636B2E004865726520796F7583
:1032F0002063616E2073656520746865206F6E2D94
:1033000073637265656E206D656E750048657265E4
:103310002061726520736F6D65206F66207468652B
:1033200020436C6F636B20446973706C6179732008
:10333000737570706F7274656400416E616C6F6755
:1033400020436C6F636B2077697468206D696E69C8
:103350006D616C206469676974730000416E616C13
:103360006F6720436C6F636B207769746820616CB2
:103370006C20646967697473000041646420746838
:103380006520323420686F757273206E756D6572BA
:10339000696320646973706C617900004F72206109
:1033A00064642074686520414D2F504D206E756D0A
:1033B0006572696320646973706C617900004D699E
:1033C0007820616E64204D61746368206173207998
:1033D0006F7520706C65617365005475726E207432
:1033E0006865204C454420626C696E6B696E67208D
:1033F0006F666600416E64207475726E2069742079
:103400006261636B206F6E005475726E206F6E2068
:1034100043616C6962726174696F6E204D6F64659F
:1034200000005475726E206974206261636B206FB6
:103430006666000054686520274127206F6E20745F
:1034400068652073636F7065206D65616E732041E0
:10345000565220436C6F636B204D6173746572200C
:103460004D6F646500004D616B652054696D65208A
:10347000676F2066617374004D616B652054696DE0
:103480006520676F206E6F726D616C004D616B65BA
:103490002054696D6520676F206261636B004D6128
:1034A0006B652054696D6520676F206261636B20D6
:1034B000666173742100566572626F7365206F7563
:1034C00074707574206973206F6E65206F66207943
:1034D0006F7572206F7074696F6E73005468652029
:1034E000626C696E6B696E67204220776F756C64E1
:1034F00020696E6469636174652061206C6F772058
:10350000525443206261636B75702062617474650C
:1035100072792C20627574206E6F7720697427731E
:10352000206A75737420612064656D6F00005468B3
:10353000697320626C696E6B696E67205020696EDA
:10354000646963617465732074686174207468656C
:10355000203120505053207369676E616C2069736D
:10356000206D697373696E672E20416761696E2CE7
:10357000206A75737420612064656D6F000057695F
:103580006C6C20746869732067657420796F75723C
:1035900020617474656E74696F6E3F004275726E5F
:1035A00020696E2070726576656E74696F6E206D2D
:1035B0006F7665732074686520646973706C6179D7
:1035C00020612074696E79206269742C206E6F729C
:1035D0006D616C6C792065766572792035206D6936
:1035E0006E757465732062757420686572652065F8
:1035F00076657279207365636F6E64005765206825
:103600006F706520796F7520656E6A6F79656420CB
:10361000746869732064656D6F2E205468616E6BE9
:1036200020796F7520666F72207573696E672074DC
:1036300068697320447574636874726F6E6978206A
:10364000436C6F636B001BA114601BA3F8940E9472
:10365000CA000E94F2000E94860178940895F3DF68
:10366000E0E0F8E350E040E06DEF73E280E05B986B
:103670005C98460F571FE81F1491012F1F7018B94F
:10368000029505B9F6CF0F930091C00005FFFCCF5E
:103690000F910093C60008958F930F9302950F70BA
:1036A000802F0E941A0C082FEEDF0F910F70802FD1
:1036B0000E941A0C082FE7DF8F91089506E40E94FC
:1036C000431B00270E944C1B082F0E944C1B072FF6
:1036D0000E944C1B062F0E944C1B0DE00E94431BB6
:1036E0000AE00E94431B08956F5F7F1D8F1D0895A0
:1036F0006C597F1D8F1D089504E6FADF0A95E9F7DE
:10370000089561507F098F09089564567F098F09D4
:10371000089504E6FADF0A95E9F708950091C600D6
:103720000E94431B0B3211F4DFDF32C0053711F466
:10373000DFDF2EC0053511F4DFDF2AC00D3211F4B2
:10374000E0DF26C0043611F4E0DF22C0043411F4B7
:10375000E0DF1EC00F3309F41BC0013319F4E0E0B1
:10376000F8E316C0023319F4E0E0F9E311C00333C3
:1037700019F4E0E0FAE30CC0043319F4E0E0FBE3F1
:1037800007C0013729F40BA10B7F0BA30E94C201D4
:0A37900095DF0F910FBF0F91189500
:10380000808386898C8F9295989C9FA2A5A8ABAE49
:10381000B0B3B6B9BCBFC1C4C7C9CCCED1D3D5D85B
:10382000DADCDEE0E2E4E6E8EAECEDEFF0F2F3F514
:10383000F6F7F8F9FAFBFCFCFDFEFEFFFFFFFFFFC9
:10384000FFFFFFFFFFFFFEFEFDFCFCFBFAF9F8F7B0
:10385000F6F5F3F2F0EFEDECEAE8E6E4E2E0DEDCC8
:10386000DAD8D5D3D1CECCC9C7C4C1BFBCB9B6B3E1
:10387000B0AEABA8A5A29F9C9895928F8C898683A9
:10388000807C797673706D6A6763605D5A575451B6
:103890004F4C494643403E3B383633312E2C2A2785
:1038A0002523211F1D1B1917151312100F0D0C0AAC
:1038B00009080706050403030201010000000000D7
:1038C00000000000000001010203030405060708D0
:1038D000090A0C0D0F1012131517191B1D1F212398
:1038E00025272A2C2E313336383B3E404346494C5F
:1038F0004F5154575A5D6063676A6D707376797C77
:10390000000102030405060708090A0B0C0D0E0F3F
:10391000101112131415161718191A1B1C1D1E1F2F
:10392000202122232425262728292A2B2C2D2E2F1F
:10393000303132333435363738393A3B3C3D3E3F0F
:10394000404142434445464748494A4B4C4D4E4FFF
:10395000505152535455565758595A5B5C5D5E5FEF
:10396000606162636465666768696A6B6C6D6E6FDF
:10397000707172737475767778797A7B7C7D7E7FCF
:10398000808182838485868788898A8B8C8D8E8FBF
:10399000909192939495969798999A9B9C9D9E9FAF
:1039A000A0A1A2A3A4A5A6A7A8A9AAABACADAEAF9F
:1039B000B0B1B2B3B4B5B6B7B8B9BABBBCBDBEBF8F
:1039C000C0C1C2C3C4C5C6C7C8C9CACBCCCDCECF7F
:1039D000D0D1D2D3D4D5D6D7D8D9DADBDCDDDEDF6F
:1039E000E0E1E2E3E4E5E6E7E8E9EAEBECEDEEEF5F
:1039F000F0F1F2F3F4F5F6F7F8F9FAFBFCFDFEFF4F
:103A000000020406080A0C0E10121416181A1C1EC6
:103A100020222426282A2C2E30323436383A3C3EB6
:103A200040424446484A4C4E50525456585A5C5EA6
:103A300060626466686A6C6E70727476787A7C7E96
:103A400080828486888A8C8E90929496989A9C9E86
:103A5000A0A2A4A6A8AAACAEB0B2B4B6B8BABCBE76
:103A6000C0C2C4C6C8CACCCED0D2D4D6D8DADCDE66
:103A7000E0E2E4E6E8EAECEEF0F2F4F6F8FAFCFE56
:103A8000FFFDFBF9F7F5F3F1EFEFEBE9E7E5E3E134
:103A9000DFDDDBD9D7D5D3D1CFCFCBC9C7C5C3C124
:103AA000BFBDBBB9B7B5B3B1AFAFABA9A7A5A3A114
:103AB0009F9D9B99979593918F8F8B898785838104
:103AC0007F7D7B79777573716F6F6B6967656361F4
:103AD0005F5D5B59575553514F4F4B4947454341E4
:103AE0003F3D3B39373533312F2F2B2927252321D4
:103AF0001F1D1B19171513110F0F0B0907050301C4
:103B000000000000000000000000000000000000B5
:103B100000000000000000000000000000000000A5
:103B20000000000000000000000000000000000095
:103B30000000000000000000000000000000000085
:103B40000000000000000000000000000000000075
:103B50000000000000000000000000000000000065
:103B60000000000000000000000000000000000055
:103B70000000000000000000000000000000000045
:103B8000FFFFFFFFFFFFFFFFFFFFFFFFFFFFFFFF45
:103B9000FFFFFFFFFFFFFFFFFFFFFFFFFFFFFFFF35
:103BA000FFFFFFFFFFFFFFFFFFFFFFFFFFFFFFFF25
:103BB000FFFFFFFFFFFFFFFFFFFFFFFFFFFFFFFF15
:103BC000FFFFFFFFFFFFFFFFFFFFFFFFFFFFFFFF05
:103BD000FFFFFFFFFFFFFFFFFFFFFFFFFFFFFFFFF5
:103BE000FFFFFFFFFFFFFFFFFFFFFFFFFFFFFFFFE5
:103BF000FFFFFFFFFFFFFFFFFFFFFFFFFFFFFFFFD5
:00000001FF
